:0200000480007A
:10000000B72F0000938F0F8073900F3015A8130047
:100010000000130000001300000013000000130094
:100020000000130000001300000013000000130084
:100030000000130000001300000013000000010086
:10004000970200009382020C73905230814001416C
:100050008141014281420143814301448144014580
:100060008145014681460147814701488148014950
:100070008149014A814A014B814B014C814C014D20
:10008000814D014E814E014F814F971102009381A6
:1000900061D1170502001305E5529795030093857A
:1000A000257A01461122170502001305A547970579
:1000B00002009385E54E0146C52817A503001305E8
:1000C000657897B503009385A57737B6ABAB130674
:1000D000B6BAD92817B103001301C176EF60E04A20
:1000E000860293D21200F512638802008242110147
:1000F0006F00001073002030824211017300203025
:10010000711116C0F3222034E3CC02FC82421101AB
:10011000130141F806C20AC40EC612C816CA1ACC88
:100120001ECE22D026D22AD42ED632D836DA3ADCC7
:100130003EDEC2C0C6C2CAC4CEC6D2C8D6CADACC97
:10014000DECEE2D0E6D2EAD4EED6F2D8F6DAFADCA7
:10015000FEDE73252034F32510340A8601A07310C7
:10016000153492402241B2414242D2426243F243AC
:10017000025492542255B2554256D2566257F25703
:10018000064896482649B649464AD64A664BF64B33
:10019000065C965C265DB65D465ED65E665FF65F83
:1001A0001301C1077300203010C16374B50011053D
:1001B000E5BF828000000000000000000000000099
:1001C000000000000000000000000000000000002F
:1001D000000000000000000000000000000000001F
:1001E000000000000000000000000000000000000F
:1001F000197106C00AC20EC412C616C81ACA1ECC8D
:1002000022CE26D02AD22ED432D636D83ADA3EDCC6
:1002100042DEC6C0CAC2CEC4D2C6D6C8DACADECC96
:10022000E2CEE6D0EAD2EED4F2D6F6D8FADAFEDCA6
:100230009702020083A2423223A02200F32210344C
:1002400096DEEF00002B170102000321E13002418E
:10025000F65273901234B72200009382028873A082
:10026000023082403242C2425243E24372448254DC
:100270001255A2553256C2565257E2577258864806
:100280001649A649364AC64A564BE64B764C865C1A
:10029000165DA65D365EC65E565FE65F0961730059
:1002A0002030970202009382E23123A0120023A2A1
:1002B000220023A4320023A6420023A8520023AA2E
:1002C000620023AC720023AE820023A0920223A21C
:1002D000A20223A4B20223A6C20223A8D20223AA06
:1002E000E20223ACF20223AE020323A0120523A2F2
:1002F000220523A4320523A6420523A8520523AADA
:10030000620523AC720523AE820523A0920723A2C7
:10031000A20723A4B20723A6C20723A8D20723AAB1
:10032000E20723ACF207EF4010531701020003214C
:10033000A1220241F65273901234B7220000938238
:10034000028873A0023082403242C2425243E243EA
:10035000724482541255A2553256C2565257E25731
:10036000725886481649A649364AC64A564BE64B45
:10037000764C865C165DA65D365EC65E565FE65FB1
:10038000096173002030970202009382A22383A0A8
:10039000020003A1420083A1820003A2C20083A243
:1003A000020103A3420183A3820103A4C20183A427
:1003B000020203A5420283A5820203A6C20283A60B
:1003C000020303A7420383A7820303A8C20383A8EF
:1003D000020403A9420483A9820403AAC20483AAD3
:1003E000020503AB420583AB820503ACC20583ACB7
:1003F000020603AD420683AD820603AEC20683AE9B
:10040000020703AFC20983AF820782807370043092
:10041000197106C00AC20EC412C616C81ACA1ECC6A
:1004200022CE26D02AD22ED432D636D83ADA3EDCA4
:1004300042DEC6C0CAC2CEC4D2C6D6C8DACADECC74
:10044000E2CEE6D0EAD2EED4F2D6F6D8FADAFEDC84
:100450009702020083A2421023A0220086DEEF2032
:10046000205A170102000321210F0241F652739016
:100470001234B72200009382028873A002308240B7
:100480003242C2425243E243724482541255A25550
:100490003256C2565257E257725886481649A649F4
:1004A000364AC64A564BE64B764C865C165DA65DD0
:1004B000365EC65E565FE65F09617300203073707A
:1004C000043001A07310453082807325403073F0F2
:1004D00043308280970700009387A7FE232EB5FE46
:1004E0002322C5FA232635F82320F5F8130505F84D
:1004F0008280411106C6EF403033EF10503601E5DF
:10050000B24041018280B24041016F20604F9307A9
:1005100085007D575CC118C55CC51CC9232005003A
:1005200082802328050082805C41DCC1984798C501
:1005300098474CC38CC788C91C4185071CC1828061
:100540009041FD57130785006314F60039A83E87D4
:100550005C439443E37DD6FEDCC18CC798C54CC395
:1005600088C91C4185071CC1828018495C43EDB7CE
:10057000584114451C4914C71845544154C3D84325
:100580006314A7001845D8C32328050088437D15A8
:1005900088C38280411122C406C626C23C412A84F7
:1005A00081EF1C41A5CF01451C5C85071CDCB240D6
:1005B0002244924441018280B2841DE608453E8671
:1005C000EF30304B1C4434405840B6971CC4E3EC29
:1005D000E7FC1C4001451CC41C5C85071CDCB240C8
:1005E000224492444101828048453E86EF30704863
:1005F00038405C4414403307E040BA975CC463F56C
:10060000D7005C403E9758C48947E39EF4F81C5CD1
:10061000D9DB1C5C0145FD171CDC79B74841EF2094
:10062000302F2322040049B7011106CE22CC26CA5E
:1006300060492AC615C0185C5C5C6365F70073707E
:10064000043001A0185C8144636BF700F2406244FF
:100650002685D244056182807370043001A02E8605
:1006600022856C00053F3844FD57AA846306F700D5
:100670003C4485073CC4D9BF5C50E9DB1305440208
:10068000EF20207A61D58544D1B73041AE8701CEC5
:100690004C455841B2954CC563E4E5000C414CC54E
:1006A0003E856F30103D8280797122D406D62A842F
:1006B00026D24AD04ECE52CC56CAEF20102E3C4401
:1006C000635CF002130A4402FD590549644889C875
:1006D000985CDC5C22C66367F7067370043001A087
:1006E0005C5099CB5285EF20C0732DED3C44FD1733
:1006F0003CC43C44E34CF0FCFD573CC4EF20302CA0
:10070000EF20B0297C406352F0021C4899CF93043B
:1007100004012685EF20E07029E97C40FD177CC0AC
:100720007C406354F0001C48EDF7FD577CC0EF207F
:100730001029B250225492540259F249624AD24AC4
:1007400045618280985CE373F7FA01466C00268568
:100750009135BC44AA8A638D3701BC448507BCC46B
:10076000E3962AF9EF20300C51B7EF20D00B75B784
:10077000DC50FDD713854402EF20A06A75D1DDB7A8
:1007800029CD011122CC2A8406CE26CA4AC84EC6DB
:100790002E89EF20902024404C5C8329040026857C
:1007A000EF5050407D57232C0402B3079540CE975D
:1007B0004E9578C048C0232434015CC438C463110A
:1007C00009021C488DE7EF20901FF2406244D2449A
:1007D0004249B2490545056182807370043001A029
:1007E000130504012D33130544021533E9BF130526
:1007F0000401EF2000638547E317F5FC0139E1B7F9
:1008000001E57370043001A0011126CA4AC84EC622
:1008100006CE22CCAA842E89B289B5C9EF50903871
:1008200013059505EF30B00C2A8425C9930785057B
:100830001CC144DC23202405EF20301624404C5CEE
:10084000032904002685EF50F035FD56232C0402C1
:10085000B30795403307A900CA9774C058C05CC459
:1008600034C4130504012324240155311305440223
:100870007939EF20D01423083405232A0404228573
:10088000F2406244D2444249B24905618280130574
:100890008005EF30D0052A8401E57370043001A093
:1008A00000C041BF797126D2AA841305800522D4E5
:1008B00006D64AD04ECE52CCEF3070032A8421C9DE
:1008C000232C0502FD577CC10547130A05013CC4D2
:1008D000528558DC23220400232004002324040032
:1008E000232604002320040423089404232A040458
:1008F0003939130944024A8519393C4002C28DC373
:100900007370043001A022854533EF101011228549
:10091000B250225492540259F249624A456182808F
:10092000EF20E07201E59247639C070AEF20F00692
:10093000185C5C5C8144FD596362F7069247C1C351
:1009400081E42800EF200061EF207007EF10E067DE
:10095000EF20B0047C4063943701232204043C441C
:100960006394370123240404EF2070054C00280011
:10097000EF20606049F9EF205002185C5C5C630373
:10098000F704EF20D00322850533EF1010098544CA
:10099000EF20B000185C5C5CE372F7FA304021E6AF
:1009A0001C40ADC701451C5C784885071CDC39CB71
:1009B00081452285953985476313F500813CEF20F9
:1009C0001000B1B7EF20A07F92455285EF2020277D
:1009D0002285D939EF1070045DF90D3C85444DBF77
:1009E0007370043001A008448145EF3090081C4426
:1009F00034405840B6971CC4E3E6E7FA1C40014572
:100A00001CC455B75C5089EB5DD94DBF4840EF2001
:100A100020702322040041BF4A85EF208040854793
:100A2000E31FF5F861BF01E57370043001A0637541
:100A3000B5007370043001A0411122C409462E8410
:100A4000814506C6753B11C500DDB2402244410117
:100A500082807370043001A0397106DE22DC26DA50
:100A60004AD84ED652D456D25AD032C66300051058
:100A70006388050E89476399F600585D85476305CD
:100A8000F7007370043001A0B6842E892A84EF2009
:100A9000005C11E5B24781C77370043001A0EF20FC
:100AA000C06F185C5C5C8149094B7D5A930A040154
:100AB0006367F706638F640BB24763890712639518
:100AC00009002808EF200049EF20606FEF10E04F89
:100AD000EF20A06C7C4063944701232204043C4433
:100AE0006394470123240404EF20606D6C00280800
:100AF000EF2060486316050EEF20206A185C5C5CEE
:100B00006302F704EF20A06B2285793EEF10E070BE
:100B10008549EF208068185C5C5CE37DF7F8304025
:100B200039CA6399040C0844CA85EF3080741C44A8
:100B300034405840B6971CC463E1E7041C400145AB
:100B40001CC42DA8EF20A067B2455685EF20200FCA
:100B50002285993EEF10606C45FD4D38854955BFA3
:100B60003C41E38907F07370043001A073700430D6
:100B700001A0304005EE1C40D5C301451C5C7848FF
:100B800085071CDC51C7A6852285793C854763040F
:100B9000F508EF20C0620545F2506254D254425924
:100BA000B259225A925A025B216182804844CA8516
:100BB000EF30206C3C4058441440B307F0403E975F
:100BC00058C46378D7005840BA975CC48947E39605
:100BD000F4FA1C5CDDD31C5C0145FD171CDC79BFFD
:100BE0002285D934EF10606301457DB7EF20205D89
:100BF00001455DB74844CA85EF30A0673C40584482
:100C00001440B307F0403E9758C4E371D7FC65BF6A
:100C10005C5099EB3DDDEFF06FFFA5BF4840EF2042
:100C2000204F2322040099BF13054402EF20601FC8
:100C30008547E310F5F6C5B70DC5411122C426C29C
:100C400006C64AC0032945002A84EF20803F81441C
:100C5000630CA900B2402244268502499244410116
:100C600082807370043001A05C448544FD175CC42D
:100C7000F5F38146014681452285F93BE1BF39CD37
:100C8000A9C9011122CC26CA4AC852C406CE4EC6F2
:100C90008947B68432892E8A2A846399F600585D82
:100CA00085476300F7067370043001A03938185C7B
:100CB0005C5CAA896367F70281444E85EFF09F80F0
:100CC000F240624426854249D244B249224A056133
:100CD00082803C41DDD77370043001A07370043012
:100CE00001A0304049E21C40DDCB1C5C7D578507EC
:100CF0001CDC3C446388E7083C44854485073CC4CD
:100D00006DBFEFF08FFC185C5C5CAA89636DF70225
:100D1000304071DA4844D285EF30A0553C40584409
:100D20001440B307F0403E9758C46375D70058404D
:100D3000BA975CC48947E39AF4FA1C5CDDD71C5C63
:100D4000FD171CDC5DB7304059DE4844D285EF30DA
:100D500040523C4058441440B307F0403E9758C4BA
:100D6000E367D7FCD9BFDDF40844D285EF3060508B
:100D70001C4434405840B6971CC4E3E8E7F61C40D6
:100D80001CC4A5B77C4895C3A685228571388544C7
:100D9000E31595F2E30309F22320990039BF484097
:100DA000EF2000372322040089B75C508544E38696
:100DB00007F013054402EF20C00669FDFDBD31CDEB
:100DC0003C4181C77370043001A01C41B1CB0111BB
:100DD00022CC26CA2A844AC84EC606CE2E89EFF0F7
:100DE000CFEE185C5C5CAA898144637DF7001C5CD3
:100DF0007D5785071CDC3C446389E7023C448544FD
:100E000085073CC44E85EFF0EFEBF2406244268547
:100E10004249D244B249056182807370043001A016
:100E20005C41D5D77370043001A07C4891CB8145DB
:100E30002285EFF06FFF8547630BF5008544D9B736
:100E40005C50EDDF13054402EF10B07D65D9E30778
:100E500009FE85472320F900D5B7397106DE22DC6B
:100E600026DA4AD84ED652D432C6630A050E6382B9
:100E7000050EB6892E892A84EF20601D11E5B24740
:100E800081C77370043001A0EF2020311C5CD1E7D2
:100E9000B247638E07102808EF20C00BFD54130AD9
:100EA000440239A8EF20A0312285EFF0EFFFEF10C8
:100EB000C036EF20802E1C5CADE3B2476389070E7D
:100EC000EF20E02FEF106010EF20202D7C40639486
:100ED0009700232204043C446394970023240404D1
:100EE000EF20E02D6C002808EF20E00855E9EF2006
:100EF000C02A1C5CC5FBEF20802C1C40BDC7B2453E
:100F00005285EF10D0532285EFF00FFAEF10E0304A
:100F100031C9EF2080281C5CCDD3CA85228544448A
:100F2000EFF0AFF6639B09041C5C1840FD171CDC56
:100F300001E7EF20402D48C01C48B9EBEF202028E6
:100F40000545F2506254D2544259B259225A216195
:100F500082803C41E38F07F07370043001A073700E
:100F6000043001A0EFF08FCA6DB7EF200023484096
:100F7000EF20E00FEF20A02459B75C5044C4DDDF20
:100F800013054402EF10F06955D9EFF02FC87DB773
:100F900013050401EF10F0688547E311F5FAF5B782
:100FA0002285EFF06FF0EF104027014559BFEF2089
:100FB0000021014579B71DC9411122C44AC006C6A6
:100FC00026C244412E892A84EF20A0076383A4020D
:100FD00081464A8681452285493585476300F50269
:100FE000B24022449244024941018280737004302D
:100FF00001A05C44054585075CC4DDB75C448507FA
:101000005CC4F9BF15CDADC9011122CC26CA4AC8AE
:101010004EC652C42A8406CE3289AE89EFF0EFCA9A
:101020001C5C2A8A814485E35285EFF0AFC9F24007
:10103000624426854249D244B249224A05618280EF
:101040007370043001A0304001CE4C445C40B29536
:101050004CC463E4F5000C404CC44E85EF30602175
:101060001C5C7D57FD171CDC7C40638CE7007C40DA
:10107000854485077CC04DBF3C41D9D7737004308F
:1010800001A01C4899E3854445B713050401EF10FE
:10109000505975D9E30909FE85472320F900E5B7C2
:1010A00021C93C41A1CDA1CB011122CC26CA4AC8FD
:1010B00052C42A8406CE4EC62E8AEFF00FC11C5CA5
:1010C0002A89814491CB8329C400D2852285EFF0FF
:1010D000CFDB8544232634014A85EFF0AFBEF240D2
:1010E000624426854249D244B249224A056182803F
:1010F0007370043001A07370043001A0EDDF7370D1
:10110000043001A001E57370043001A0411122C434
:101110002A8406C6EF206008005CEF20400AB24037
:10112000228522444101828001E57370043001A0D0
:10113000411106C622C42A84EF2020061C5C405CB4
:101140001D8CEF20C0072285B240224441018280DD
:1011500019C1085D82807370043001A01DCD97878E
:1011600003009387276AD843630CE502D847630CD2
:10117000E504D84B6307E504D84F6302E504D85370
:10118000630DE502D8576308E502D85B6303E50207
:10119000D85F630EE5006F30A0077370043001A0C4
:1011A00001470E07BA9723A007006F3060061D475E
:1011B000CDBF1947FDB71547EDB71147DDB70D474F
:1011C000CDB70947F9BF0547E9BF684582806CC5BF
:1011D000828003450505828009C5085D1335150029
:1011E00082807370043001A019C51C5D485D1D8D9F
:1011F0001335150082807370043001A097870300B7
:1012000093874760984305C3984705C7984B05C720
:10121000984F05C7985305C7985705C7985B15C7DA
:10122000985F15C3828001470E07BA978CC3C8C365
:1012300082800547D5BF0947C5BF0D47F5B71147A0
:10124000E5B71547D5B71D47C5B71947F1BF97870C
:1012500003009387275BD8436308E502D847630BF5
:10126000E502D84B630AE502D84F6309E502D8537B
:101270006308E502D8576307E502D85B6308E50217
:10128000D85F6303A702828001470E07BA9723A0A5
:10129000070082800547D5BF0947C5BF0D47F5B791
:1012A0001147E5B71547D5B71D47C5B71947F1BF72
:1012B000797122D426D24AD02A8406D64ECE52CC78
:1012C00056CAAE843289EF10506D7840FD576314D2
:1012D000F700232204043844FD576314F700232445
:1012E0000404EF10D06D1C5C99E74A86A6851305AF
:1012F0004402EF10D027EF10506A3C44635CF002C8
:10130000130A4402FD590549644889C8985CDC5CAD
:1013100022C66367F7067370043001A05C5099CB56
:101320005285EF10103035ED3C44FD173CC43C4471
:10133000E34CF0FCFD573CC4EF107068EF10F06513
:101340007C406352F0021C4899CF93040401268527
:10135000EF10302D31E97C40FD177CC07C40635498
:10136000F0001C48EDF7FD577CC0EF105065B250FF
:10137000225492540259F249624AD24A456182800B
:10138000985CE373F7FA01466C002685EFF08FA0B6
:10139000BC44AA8A638D3701BC448507BCC4E3956D
:1013A0002AF9EF10504849B7EF10F0476DB7DC50FD
:1013B000FDD713854402EF10D02675D1DDB701E5C6
:1013C0007370043001A0411126C2AA840A051305D6
:1013D000950522C406C64AC0EF2070512A843DC13B
:1013E000930785051CC191473CC144DDEF10F05ABD
:1013F00024404C5C032904002685EF40B07AFD565A
:10140000232C0402B30795403307A900CA9774C080
:1014100058C05CC434C41305040123242401EFF034
:101420000F8F13054402EFF08F8EEF1050592308F1
:101430000404232A04042285B2402244924402492F
:10144000410182807370043001A0411122C426C280
:101450004AC02A8406C62E89EF1030547C48814445
:1014600091CBEF10D055B2402244268502499244D8
:10147000410182801C5C8144EDF7232A24058544C8
:10148000CDB77C496385B70081473E858280185D72
:10149000814765FF411122C42A8406C6EF10F04F30
:1014A000232A0404EF10B051B240224485473E8500
:1014B0004101828001112E8681466C0006CE02C653
:1014C000693AF240324505618280011106CE22CC94
:1014D00026CA02C605C12A84EFE03FFF1C5CAA842D
:1014E00089EF2685EFE01FFEF24062443245D24488
:1014F000056182807370043001A0304001CE4C44FD
:101500005C40B2954CC463E4F5000C404CC46800E8
:10151000EF2030561C5C7D57FD171CDC7C40638639
:10152000E7007C4085077CC06DBF1C48DDDB1305F0
:101530000401EF10100F75B71DC179714ECE52CC5A
:1015400006D63E8A22D426D24AD056CA5AC85EC689
:10155000A547BA8963F8E7007370043001A073707F
:10156000043001A02A8BAE843289B68BC28A63070D
:10157000082213050006EF2090372A84630B05200C
:101580000A09232855034A869305500A5685EF20F9
:10159000505C03C704001C587119230AE40203C7F6
:1015A00004003E991379C9FF79C783C71400A30AC1
:1015B000F40283C71400E1C383C72400230BF402A1
:1015C00083C72400CDCB83C73400A30BF40283C7A9
:1015D0003400D5C383C74400230CF40283C74400FE
:1015E000D9CB83C75400A30CF40283C75400C1C7EE
:1015F00083C76400230DF40283C76400ADCF83C7A3
:101600007400A30DF40283C77400B5C783C78400B8
:10161000230EF40283C78400B9CF83C79400A30EBE
:10162000F40283C79400A1CB83C7A400230FF40264
:1016300083C7A400A9C383C7B400A30FF40283C760
:10164000B40095CB83C7C4002300F40483C7C4004F
:101650009DC383C7D400A300F40483C7D40081CF03
:1016600083C7E4002301F40483C7E40089C783C768
:10167000F400A301F404930A44005685A301040472
:101680002326340323283405232A0404EFE07FE9CA
:1016900013058401EFE0FFE8A947B3873741232C06
:1016A000040400C81CCC40D023220404232E0404CC
:1016B0005E86DA854A85EFE0FFE108C063040A0030
:1016C00023208A007370043017F90100130909E719
:1016D0008327090097F40100938404E891C7984098
:1016E0009C407C4385077CC317F701001307C7E5BF
:1016F0001C43850797F6010023A8F6E49C40C5CB60
:101700008327090017FB0100130B8BF389EB9C4027
:10171000DC5763E6F90097F7010023AF87E297F7FC
:1017200001009387A7E09C4317F70100130747E1E7
:1017300048541843850797F6010023A9F6DE3CC4F8
:101740006376A70097F7010023ACA7DED145EF40F1
:101750007045D6855A95EFE03FDD8327090081C7A4
:101760009C40FC43B5E383270900054499C79C408E
:10177000DC5763F43701EFE07FC92285B250225471
:1017800092540259F249624AD24A424BB24B4561E5
:1017900082805685EF20D0277D54C5B713152600CB
:1017A000EF20F014AA8AE31605DC7D54F9B797F709
:1017B000010023A387DA184385476301F70217FB6B
:1017C0000100130BEBE7A1BF984094407C43FD1749
:1017D0007CC3FC42C9FB7360043071B7014A17FB3C
:1017E0000100130BEBE5A94B5285D145EF40903B2F
:1017F000050A5A95EFE0BFD1E3187AFF97FB010085
:10180000938B8BF05E85EFE09FD017FA0100130AEF
:10181000EAF05285EFE0BFCF17F50100130545F15F
:10182000EFE0FFCE17F501001305C5F1EFE03FCE65
:1018300017F50100130545F2EFE07FCD97F70100A2
:1018400023AA77D197F7010023A447D1C9BD41113D
:1018500022C406C626C24AC02A847370043097F494
:1018600001009384A4CD9C40F9E311E497F70100B3
:10187000938787CE8043130944004A85EFE05FCF0A
:101880001C5489C713058401EFE09FCECA8517F564
:101890000100130525EBEFE03FC997F7010093879F
:1018A000E7CA984397F70100938747C89C43050709
:1018B00097F6010023ACE6C89840850797F601002B
:1018C00023A6F6C601CB97F701009387E7C8984394
:1018D000784349EF9C40B1C797F701009387C7C78A
:1018E0009843630F870873700430984039EB17F7FB
:1018F0000100130727C614439442A5E27D5797F6CB
:10190000010023A3E6C2984009CF9843784311CB46
:10191000984394437C43FD177CC3FC4299E3736076
:101920000430B2402244924402494101828097F738
:101930000100938767C298439C437C4385077CC31F
:101940002DB794439843F8420507F8C217F70100F2
:10195000130747C014439442D5D2184358475847F9
:10196000584397F6010023A1E6BC71BF9843944306
:101970007C43FD177CC3FC42B1FF7360043099BF08
:1019800097F70100938707BA9C4381C773700430AF
:1019900001A02244B2409244024941016FE01FA7D6
:1019A00041C517F70100130727BB14438147638B19
:1019B000A606411106C622C426C27370043097F6EB
:1019C00001009386A6B79C4291C710431C437C42FA
:1019D00085077CC29C42AA84404981C71C43FC43C2
:1019E000B9E797F701009387E7B69C43638B8704B9
:1019F00097F701009387C7B59C436384870497F7E3
:101A00000100938767D56309F40297F70100938774
:101A100067D36301F4028547B240224492443E8575
:101A2000410182803E8582807370043001A0EF40C6
:101A3000302B45BF9147CDB79C5493B7170089070A
:101A4000E1BF8947D1BF7370043097F701009387D6
:101A5000E7AE984309EF15C59C43485581CB97F7EE
:101A60000100938767AF9843784315E3828017F7A7
:101A70000100130767AE14431843F8420507F8C284
:101A800061FD17F70100130727AD0843F1B798432D
:101A900094437C43FD177CC3FC42E9FB7360043034
:101AA0008280411122C42A8406C6EFE01FA211E4FD
:101AB00097F70100938747AA80434054EFE09FA027
:101AC000B2402285224441018280A54763F5B700D8
:101AD0007370043001A0011122CC06CE26CA4AC878
:101AE0004EC652C42A847370043017F901001309DA
:101AF000E9A483270900CDEF71C43C486388F50849
:101B000017F70100130747A563FCB7001443638C64
:101B1000860C18434457B3B4950093C4140029A00D
:101B20000443818C93B4140058546383E70A1C4C1B
:101B30002CC863C60700A947B385B7400CCC9317E0
:101B40002700BA97584897F90100938969AF8A0727
:101B5000CE97631AF702130A44005285EFE05FA1A3
:101B600097F701009387C79D48549C4363F6A700ED
:101B700097F7010023A6A79CD145EF40B002D2857C
:101B80004E95EFE07F9A99C0EFE05F8883270900C8
:101B900081CB97F701009387279C9C43FC439DEBE7
:101BA000F2406244D2444249B249224A05618280ED
:101BB00097F701009387479A98439C437C43850796
:101BC0007CC305FC97F7010093870799804335B7DD
:101BD0004CD4B1BF6244F240D2444249B249224A95
:101BE00005616F40F00F814481B725C1011126CAFC
:101BF00097F40100938444969C4006CE22CC4AC8B8
:101C00004EC6638DA7027370043017F901001309E3
:101C1000E9928327090091C798409C407C4385073F
:101C20007CC3584997F70100938707B36302F70213
:101C30008327090081C79C40FC43A5EBF240624426
:101C4000D2444249B249056182807370043001A0D8
:101C50001C5517F701001307A7ADE38BE7FCE9FB61
:101C6000930945002A844E85EFE09F9097F7010085
:101C70009387078D48549C4363F6A70097F70100AC
:101C800023A0A78CD145EF40E07197F7010093871F
:101C9000279B3E95CE85EFE03F899C405854DC570A
:101CA000E368F7F8EFE08FF661B76244F240D244A0
:101CB0004249B24905616F40B00215CD011122CCF5
:101CC00026CA4EC62A8406CE4AC8EFE01F8058486E
:101CD00097F70100938747A8AA8981446300F70218
:101CE0004E85EFE02FFEF240624426854249D24401
:101CF000B249056182807370043001A01C5417F54D
:101D000001001305E5A2E38DA7FCF9FB97F701009D
:101D1000938747819C43A9EB97F701009387C7837B
:101D20009C43445413094400DC574A85B3B4F4007F
:101D3000EFE01F8497F701009387878048549C4306
:101D400093C4140063F6A70097E7010023AAA77EB7
:101D5000D145EF40206597F701009387678ECA85CC
:101D60003E95EFE06FFCADBF93058401EFE0CFFB44
:101D700085BF0111056506CE22CC26CA4AC84EC6CB
:101D800052C456C25AC0EF208036630E051AAA8488
:101D900013050006EF20A0352A84630A051C05669A
:101DA0009305500A04D92685EF20A05A0458856768
:101DB000F117BE94B7474C4593879744130A4400E4
:101DC0005CD85285230C0402A301040423260402D8
:101DD00023280404232A0404EFE0AFF4130584014C
:101DE000EFE02FF4A947232C0404F19800C81CCC81
:101DF00040D023220404232E04040146971500003A
:101E00009385E5B12685EFE0EFEC08C073700430F0
:101E100017E90100130989728327090097E401007B
:101E20009384847391C798409C407C4385077CC30E
:101E300017E70100130747711C43850797E6010068
:101E400023A4F6709C40C9C38327090097E90100C9
:101E50009389097F81EB9C40DC5789E797E7010074
:101E600023AC876E97E701009387476C984397E60A
:101E700001009386E66C5C549442050717E6010066
:101E80002326E66A38C463F6F60017E70100232923
:101E9000F76A139527003E950A05D2854E95EFE027
:101EA000AFE88327090081C79C40FC43DDE7832717
:101EB000090091C39C40EF10F04985476305F50C7C
:101EC00059E17370043001A097E7010023A68768E9
:101ED0001843854797E9010093898976E314F7F859
:101EE000CE8A17FB0100130B2B825685D10AEFE037
:101EF0000FE2E31C5BFF17F501001305E580EFE03F
:101F00000FE197FA0100938A6A815685EFE02FE08E
:101F100017F501001305C581EFE06FDF17F501002C
:101F200013054582EFE0AFDE17F501001305C5820A
:101F3000EFE0EFDD97E7010023AE676197E701006F
:101F400023A8576105B7F2406244D2444249B249DE
:101F5000224A924A024B05618280984094407C4319
:101F6000FD177CC3FC42A1F77360043089B762445B
:101F7000F2404249B249224A924A024B2685D24453
:101F800005616F20E02873700430FD5717E70100EA
:101F9000232CF758624497E7010023A1A75AF24087
:101FA000D2444249B249224A924A024B97E7010081
:101FB00023AA075805616FE0CFAE7370043097E72E
:101FC000010023AD07566FE00FBC17E701001307B0
:101FD00067551C4385071CC382807370043097E7E4
:101FE00001009387A755984305E317E701001307FE
:101FF000675508439C4381CB97E701009387C755FA
:102000009843784301EF828017E701001307C75414
:1020100014431843F8420507F8C2C1BF98439443DC
:102020007C43FD177CC3FC42F9FF7360043082805F
:10203000411106C622C4EFE04FC997E7010093871C
:1020400067508043EFE00FC8B2402285224441012F
:10205000828097E701009387274F884382807971B8
:1020600006D622D426D24AD04ECE52CC56CA5AC810
:102070005EC697E701009387E74A9C43B1EF17E7F5
:1020800001001307274C1C43850797E6010023AB8B
:10209000F64A832A0700638F0A0697E701009387B1
:1020A000A7489C43814463F1FA0897E901009389AA
:1020B000295917EA0100130A2A4A83270A0085468C
:1020C000D85793172700BA978A07BE9983A70900A4
:1020D00063FFF600854421A897E701009387C74571
:1020E0009C438144850717E701002327F74497E7BE
:1020F0000100938727449C4391C38544B2502254E6
:10210000268502599254F249624AD24A424BB24B56
:102110004561828017E401001304C4431C409C43C2
:10212000DDC37370043001A017E40100130484427E
:1021300097E901009389C95017EA0100130ACA41BF
:1021400017EB0100130BCB3F1C409C43B5C31C4055
:10215000DC4703A9C70083274900930B49005E852C
:1021600063EEFA04EFE0CFC08327890213058901EB
:1021700099C3EFE0EFBF8327C90203270B00DE8579
:10218000139527003E950A054E956376F70017E7ED
:1021900001002327F73AEFE02FB983270A0003272E
:1021A000C902DC57E362F7FA1C4085449C43C5F33F
:1021B000FD5717E701002329F73601B717E701009C
:1021C0002324F736DDBD17E70100130767381C40ED
:1021D000184397E6010023AFE63617E701002329ED
:1021E000F73697E701009387A7349C43850717E7E5
:1021F0000100232FF7321C409C4399E7FD5717E756
:1022000001002323F73251BD1C40DC47DC47DC438F
:1022100017E70100232AF73049B597E701009387B4
:102220006730984301E77370043001A0011106CEB6
:1022300022CC26CA4AC84EC652C456C25AC073706F
:10224000043097E401009384642F984061EB984335
:102250007D1797E6010023A7E62C9C43D9EB97E76F
:1022600001009387672E9C43C9C797EA0100938AB0
:102270002A3D17EA0100130AAA2C17E901001309E5
:10228000A92D854919A83385EA00EFE0EFA9832736
:1022900009005854DC576379F70483A70A0FC1CFAC
:1022A00083A7CA0FC04713058401EFE06FAC130B7F
:1022B00044005A85EFE0CFAB5C5483260A00DA85F0
:1022C000139527003E950A052A875695E3FDF6FAF1
:1022D00017E701002326F726EFE00FA58327090063
:1022E0005854DC57E36BF7FA97E7010023A437252E
:1022F0006DB701449C4081CB97E701009387C725C8
:102300009C43FC4395E72285F2406244D244424913
:10231000B249224A924A024B0561828017E70100C6
:102320001307872314431843F8420507F8C205B77B
:10233000EF40001BC9BF17E401001304E41F1C4059
:1023400095C31C40054999CF193B09C597E7010082
:1023500023A2271F1C40FD1717E70100232EF71C9F
:102360001C40FDF397E701009387C71C98438547FE
:10237000E311F7F8EFE08F890544ADBF11CD81E59A
:102380007370043001A017E701001307A7191C435D
:1023900099C77370043001A07370043001A041111B
:1023A00022C406C614431841850617E60100232BF4
:1023B000D61697E601009386E61894423304B700D8
:1023C00000C163F7E602637FE40063FD860097E7E0
:1023D00001009387671888431105EFE06F99228504
:1023E000EF40C0091D3D01C9B24022444101828035
:1023F000E36FE4FCD9BF2244B24041016FE00F819A
:1024000011C917E701001307E7111C4391C7737047
:10241000043001A06FD09FFF411106C622C41843AB
:10242000AA87050797E6010023AEE60E97E60100AE
:102430009386861217E701001307C71018438842D6
:102440003304F7001105EFE0AF922285EF4000035F
:10245000E93311E52244B24041016FD03FFBB24065
:10246000224441018280411122C406C697E701003F
:102470009387470B9C430144850717E701002323FB
:10248000F70A97E701009387270C9C4363E0F51256
:1024900017EE0100130E8E2697E201009382821937
:1024A00001440147854F1303500A21A0311E638D5B
:1024B000C20B83278EFFBA86F5DB8327CEFFDC4372
:1024C000232EFEFE638AC70F03AFC700DC432A97A3
:1024D000814E232EFEFE6385C70783A8C70093871E
:1024E0004803232017015CC383A788042326F70130
:1024F0001CC783A7C8021CCB83A70805232C070091
:102500005CCB03A808038347080063906704C28775
:10251000850783C60700B3850741E38B66FE898183
:10252000C205C181231EB700850E1307070263068B
:102530001F038327CEFFDC43232EFEFEE39FC7F954
:1025400083274E00232EFEFE49BF8145231EB70080
:10255000850E13070702E31E1FFD76941317540020
:10256000311EBA86E397C2F597E70100938787FE8D
:1025700003AE070083270E00639D070E97E7010057
:10258000938707FD03AE070083270E0063920718A9
:1025900017EE0100130ECE0A83274E109DE383270A
:1025A0008E116395072019C223200600BD312285B4
:1025B000B24022444101828083274E00232EFEFE3A
:1025C00021B783278E1017EF0100130F2F18DC435C
:1025D00017E70100232AF7166380E73383A2C700B9
:1025E000DC43AA96814E17E70100232FF714914F81
:1025F0001303500A6388E70783A8C700938748033B
:1026000023A01601DCC283A7880423A6F6019CC67A
:1026100083A7C8029CCA83A7080523AC0600DCCAAE
:1026200003A80803834708006391672AC2878507C8
:1026300003C70700B3850741E30B67FE93D7250067
:10264000C207C183239EF600850E93860602638629
:10265000122983278E10DC4317E701002326F70E8B
:10266000E39CE7F983270E1117E70100232EF70CEF
:1026700061B783274E00130F8E00D4432322DE0060
:102680006388E629B307E500D84283A2C600814EDD
:102690002322EE00894F1303500A6306EF068328B6
:1026A000C7001387480323A01701D8C303A78804D2
:1026B00023A6F70198C703A7C80298CB03A708056C
:1026C00023AC0700D8CB03A808030347080063180E
:1026D000671C4287050783460700B3050741E38B64
:1026E00066FE13D7250042074183239EE700850E2F
:1026F00093870702638D121B83264E00D842232244
:10270000EE00E31EEFF80327CE002322EE0041BFC8
:1027100083274E00130F8E00DC432322FE006384C8
:10272000E71F83A2C700DC43AA96814E2322FE0046
:10273000894F1303500A6306FF0683A8C7009387D7
:10274000480323A01601DCC283A7880423A6F60150
:102750009CC683A7C8029CCA83A7080523AC0600B1
:10276000DCCA03A808038347080063966710C28782
:10277000850703C70700B3850741E30B67FE93D7BF
:102780002500C207C183239EF600850E93860602AC
:10279000638B120F83274E00DC432322FE00E31ECF
:1027A000FFF88327CE002322FE0041BF8327CE11EE
:1027B00097EE0100938ECEFADC4317E70100232F3A
:1027C000F7F86384D71383AFC700DC433307D50022
:1027D000014397E6010023A3F6F80D4F89429308C1
:1027E000500A6387D707C8479307450308C35CC3EC
:1027F0003C452326E7011CC75C551CCB1C5599C3DF
:10280000232657003C49232C07005CCB03280503F3
:102810008347080063951705C287850783C60700AD
:10282000B3850741E38B16FF93D72500C207C18309
:10283000231EF700050313070702638AAF028327ED
:10284000CE11DC4397E6010023AAF6F0E39DD7F909
:1028500083274E1297E6010023A2F6F069B781475D
:10286000231EF700050313070702E39AAFFC1A942F
:10287000E31C06D225BB8147239EF600850E938676
:102880000602E39912F117EE0100130E6EDB8327A7
:102890004E10769493165400E38307D01DB301477E
:1028A000239EE700850E93870702E39712E597E7DB
:1028B00001009387E7C903AE07007694931654008E
:1028C00083270E00E38607CCA1B58147239EF6003F
:1028D000850E93860602E39E12D783278E11769487
:1028E00093165400E38107CCD1B583274E1217E726
:1028F00001002325F7E6C1BD83270E1117E701006C
:102900002324F7E4E1B98327CE002322FE0011BD82
:102910008326CE002322DE00B5B3797126D24AD0B9
:102920004ECE52CC56CA5AC85EC606D622D497E9B5
:102930000100938929BF17E90100130969D017EA3B
:102940000100130AAABF97EA0100938AEAC097EB35
:102950000100938B6BBF97E40100938424BF054B68
:1029600021A883A7090003244910850717E7010060
:10297000232AF7BA5D3011E89C40E5F78327090068
:10298000E37CFBFEEFD09FA8C5BF737004308327A4
:102990000A00B9E383270911C04713054400EFD0AB
:1029A0003FBD83A70B00FD1717E70100232EF7B8E3
:1029B0009C40FD1717E70100232AF7B883270A0078
:1029C00089C783A70A00FC4385E30858EF10500429
:1029D0002285EF10F0034DB703A70A0083A70A0072
:1029E0007C4385077CC37DB703A70A0083A60A0042
:1029F0007C43FD177CC3FC42E9FB73600430F1B7F4
:102A000097E70100938707B29C43DDE7411106C6B3
:102A100022C426C297E7010023AE07B017E70100E2
:102A2000130787B31C43B7A6A5A59386565A9C5B8C
:102A30008C43639BD500D0436318B60094476395DD
:102A4000C600DC476388D70008430C4393854503E1
:102A5000EF20E07817E70100130787AE144317E46F
:102A600001001304E4BD11A81C43A9CF1C43FD17AA
:102A700097E6010023A6F6AC144393972600B69779
:102A80008A07A2979C43EDD3084393172500AA9782
:102A90008A073307F4005443A107A297C44244C3F2
:102AA0006385F402DC44B240224417E70100232589
:102AB000F7AA924441018280854717E70100232B42
:102AC000F7A682807370043001A0C440D145EF3076
:102AD000700D229544C1F9B701114AC806CE22CC27
:102AE00026CA4EC62A897370043097E40100938485
:102AF000E4A49C4017E40100130404A6D9E763147E
:102B0000090003290400930949004E85EFD05FA610
:102B10008327890289C713058901EFD07FA5CE8558
:102B200017E50100130545C3EFD01FA09C4081C7E6
:102B30001C40FC43ADE31C40638B27079C409DCFAA
:102B4000737004309C40C1EB97E70100938787A026
:102B50009843184325EBFD5717E701002326F79C00
:102B60009C4089CF1C40FC4391CB184014407C43CF
:102B7000FD177CC3FC4299E373600430F240624469
:102B8000D2444249B2490561828018401C407C43CE
:102B900085077CC3ADB7184014407C43FD177CC348
:102BA000FC42D1FB736004301C40E39927F99C4040
:102BB000A1C397E701009387E7969C43ADCB737061
:102BC000043001A09C43DC47DC47DC4317E70100ED
:102BD000232CF79471B718401C407C4385077CC3B5
:102BE00097E7010093870797984318432DD7D9BFDC
:102BF00097E701009387479517E70100130747A45C
:102C00009C4303278711631DF700F240624497E756
:102C1000010023A30794D2444249B249056182804E
:102C20006244F240D2444249B2490561D1BB624498
:102C3000F240D2444249B24905616FD02FFD3DC9EF
:102C4000411126C297E40100938404914AC02E8961
:102C50008C4006C622C4E105EFD09F8E8840110546
:102C6000EFD01F91FD57630AF90497E7010093879E
:102C7000678D804398409C434A9440C3636CF4043E
:102C800097E701009387078D88438C409105EFD02B
:102C90003F8B97E70100938727899C436376F40075
:102CA00097E7010023A28788B24022449244024958
:102CB000410182807370043001A08C402244B240F4
:102CC0009244024917E50100130505A99105410148
:102CD0006FD09F8597E701009387878788432244B9
:102CE0008C40B24092440249910541016FD05F850A
:102CF00011C997E701009387E7829C4399E77370B6
:102D0000043001A07370043001A0411126C297E481
:102D10000100938464849840AE878C40B70600809D
:102D2000D58F06C622C41CCFE1053284EFD0CFFF79
:102D300088401105EFD0DF83FD57630EF40097E75D
:102D40000100938727808843B24092442295224411
:102D500041016F30A0728C402244B240924417E58A
:102D600001001305659F910541016FD0EFFB25CD53
:102D7000411126C297D401009384047E4AC02E8953
:102D80008C4006C622C4E1053284EFD0EFF98840BA
:102D90001105EFD0EFFD8547630AF40497D70100D2
:102DA0009387477A804398409C434A9440C3636C1E
:102DB000F40497D701009387E77988438C40910505
:102DC000EFD00FF897D70100938707769C4363767F
:102DD000F40097D7010023A98774B240224492449B
:102DE0000249410182807370043001A08C4022446A
:102DF000B2409244024917E501001305E59591059B
:102E000041016FD06FF297D70100938767748843B1
:102E100022448C40B24092440249910541016FD056
:102E20002FF2411106C622C426C25C45C04735CCEC
:102E3000930484012685EFD0AFF397D701009387E1
:102E4000676E9C43B5E7930444002685EFD04FF2AC
:102E500097D701009387C76E58549C4363F6E700E9
:102E600097D7010023AEE76C93172700BA978A071C
:102E700017D501001305C57CA6853E95EFD0CFEA96
:102E800097D701009387476D9C4358540145DC5701
:102E900063F8E700854717D70100232DF76805453C
:102EA000B24022449244410182807370043001A0F8
:102EB000A68517E501001305A587EFD0EFE6C9B792
:102EC00097D70100938707669C4381E773700430AE
:102ED00001A0411106C622C426C2B70700804045A2
:102EE000CD8F1CC12DC4EFD0AFE8930444002685DC
:102EF000EFD00FE897D701009387876458549C431D
:102F000063F6E70097D7010023ACE7629317270029
:102F1000BA978A0717D50100130585723E95A685D5
:102F2000EFD08FE097D70100938707639C435854F5
:102F30000145DC5763F8E700854717D70100232BCD
:102F4000F75E0545B240224492444101828073708D
:102F5000043001A011CD97D701009387675D984396
:102F600097D701009387075E9C4318C15CC182809C
:102F70007370043001A055C1D1CD411106C622C4E1
:102F80002A877370043097D801009388285B83A741
:102F9000080091CB97D701009387075C94439C432B
:102FA000FC428507FCC217D301001303A3599C41BF
:102FB00003260300FD560144638FD70217DE01008C
:102FC000130E0E5703250E00032807005443630514
:102FD000A80005446371D6023308D6400544637CDB
:102FE000F80003250E00918F03260300B6979CC1BD
:102FF00008C350C3014483A7080081CB97D70100C1
:10300000938787559C43FC4381EF2285B24022443D
:10301000410182807370043001A07370043001A0FC
:10302000EF30004CDDB7854717D701002324F75058
:10303000828019C1684582800145828011C16CC5BA
:10304000828097D70100938727518843828097D742
:1030500001009387A74E9C43054589CB97D7010074
:103060009387474C8843133515000605828031CD80
:10307000011126CA97D401009384044E9C4006CEC9
:1030800022CC4AC84EC65855DC576379F7021C4D0E
:1030900063C707009C40D457A947958F1CCD931751
:1030A0002700BA97584917D90100130969598A07A7
:1030B000CA97630DF7009C40DC575CD5F240624430
:1030C000D2444249B2490561828082809309450019
:1030D0002A844E85EFD0CFC99C4017D70100130733
:1030E00027461843DC575CD46376F70017D70100F6
:1030F0002328F744139527003E9562440A05F240C1
:10310000D244CE854A95B249424905616FD0CFC1BC
:1031100019CD411106C622C426C297D70100938754
:10312000A74380436307A4007370043001A00145E6
:1031300082807C4881E77370043001A05454384881
:10314000FD177CC86383E60099C70145B24022445D
:10315000924441018280930444002685EFD04FC100
:10316000284897D701009387A73D9843A947898F9F
:1031700048D41CCC6376A70097D7010023A2A73CB4
:10318000D145EF30202297D701009387674B3E95BA
:10319000A685EFD06FB9054555BF7370043097D73A
:1031A00001009387A7399C4391CB97D70100938760
:1031B000A73A98439C437C4385077CC3828097D77A
:1031C00001009387A7379C438DC397D7010093874E
:1031D000A7389843784311CB984394437C43FD1719
:1031E0007CC3FC4299E373600430828097D701006E
:1031F00093878736904394439843A947D456084E03
:10320000958F1CCF828097D701009387E73498432E
:1032100009C79443F84A0507F8CA88438280797140
:103220004AD006D622D426D24ECE2A8973700430D4
:1032300097D40100938484309C4017D40100130478
:10324000A431BDE31C40BC4F89E71C400547F8CFC3
:10325000D1E19C4081C71C40FC43F1EB737004300A
:103260009C408DEF1C40A84F11C5630409021C400F
:1032700023AC07041C4023AE07049C4081C71C40BC
:10328000FC438DEBB250225492540259F2494561ED
:10329000828018403C4FFD173CCFE9BF18401C40CE
:1032A0007C4385077CC37DBF18401C407C43850759
:1032B0007CC349BF184014407C43FD177CC3FC42CB
:1032C000F1F373600430B250225492540259F2491F
:1032D0004561828008402EC61105EFD06FA9B24526
:1032E000FD576380F50697D701009387A72583A92B
:1032F000070018409C43AE992322370163ECF90480
:1033000097D701009387072588430C409105EFD09C
:103310002FA397D70100938727219C4363F6F900D9
:1033200097D7010023A23721EFD04F8E1DB7184049
:1033300014407C43FD177CC3FC428DF37360043062
:1033400031BF0C4017D50100130505419105EFD0A1
:10335000AF9DD9BF97D701009387871F88430C4043
:103360009105EFD0EF9DC9B779714AD04ECE06D600
:1033700022D426D252CC2E89B2897370043097D4CD
:1033800001009384A41B9C4017D401001304C41CA7
:10339000F9EF18408947784F630CF7001C4013453C
:1033A000F5FFB84F798DA8CF1C400547F8CFADE6A3
:1033B0009C4081C71C40FC43F5E3737004309C4083
:1033C000B1E7638609001C40BC4F23A0F9001840F8
:1033D00085470145784F630BF7001C401349F9FFFF
:1033E0000545B84F3379E90023AC27051C4023AECF
:1033F00007049C4081C71C40FC43C1E3B2502254E7
:1034000092540259F249624A4561828018401C4038
:103410007C4385077CC375B7084036C61105EFD0DD
:103420002F95B246FD576385F60897D7010093871D
:10343000671103AA070018409C43369A23224701CC
:103440006363FA0897D701009387C71088430C403D
:103450009105EFD0EF8E97D701009387E70C9C433F
:103460006370FA0697D7010023A0470D91A8184072
:103470001C407C4385077CC329BF184014407C4313
:10348000FD177CC3FC42BDFB73600430B250225474
:1034900092540259F249624A4561828018401440B0
:1034A0007C43FD177CC3FC4289FB7360043031B759
:1034B0000C4017D501001305252A9105EFD0CF86C2
:1034C000EFC0DFF4F5B597D701009387670888430D
:1034D0000C409105EFD0CF86E5B751C1411106C62A
:1034E00022C426C24AC07370043097D4010093846A
:1034F000E4049C40B9EB99C23C4D9CC2B28789461A
:10350000704D74CD2E872A846386D70663FCF6043B
:103510008D456387B70091456395B7006300D60C6E
:1035200038CC8547630FF60405449C4081CB97D780
:103530000100938767029C43FC43A9E32285B240C4
:103540002244924402494101828097D70100938727
:10355000A70098439C437C4385077CC369BF737075
:10356000043001A08546E39ED7FA3C4D33E7B7000F
:1035700038CD45BF3C4D85073CCD65B7EF20507633
:1035800075BF130944004A85EFC09FFE97D701001D
:10359000938707FB48549C4363F6A70097D7010025
:1035A00023A0A7FAD145EF20F05F97D701009387BA
:1035B00027093E95CA85EFC03FF71C5481C7737039
:1035C000043001A097D70100938707F99C43585412
:1035D000DC57E3FBE7F4EFC07FE3B9B70144B1B7D1
:1035E00039CD011122CC26CA4AC84EC652C456C291
:1035F00006CEBA89368AB2842E892A84EFC0FFECBF
:10360000AA8A63050A003C4C2320FA00784C8947BB
:103610007CCC6389F40263F4970C8D466387D400F5
:1036200091466396D400630AF70A232C2405854744
:10363000631EF7061C5499CB7370043001A073709D
:10364000043001A03C4C85073CCCD5B797D701008E
:10365000938747ED9C43ADEB930444002685EFC070
:103660003FF197D701009387A7ED48549C4363F639
:10367000A70097D7010023A5A7ECD145EF209052D2
:1036800097D701009387C7FBA6853E95EFC0DFE97A
:1036900097D70100938747EC9C435854DC5763F756
:1036A000E70063850900854723A0F9000544568596
:1036B000EFC05FE12285F2406244D2444249B24900
:1036C000224A924A056182809305840117D5010040
:1036D00013050506EFC05FE565BF0144C9BF854717
:1036E000E397F4F43C4C33E92701232C240581B7FC
:1036F0004DC1011122CC26CA2A844EC606CE4AC824
:10370000AE84EFC09FDC8947744C7CCC3C4C0547B1
:10371000AA8985073CCC6395E6061C5481C7737063
:10372000043001A097D701009387C7DF9C43ADE722
:10373000130944004A85EFC0BFE397D70100938780
:1037400027E048549C4363F6A70097D7010023A9BC
:10375000A7DED145EF20104597D70100938747EEAC
:10376000CA853E95EFC05FDC97D701009387C7DE1F
:103770009C435854DC5763F5E70099C085479CC0CB
:103780006244F240D24442494E85B24905616FC05D
:103790007FD37370043001A09305840117D5010015
:1037A000130505F9EFC05FD8C1B7AA8729C57370A3
:1037B000043017D70100130767D814439DE2F04F78
:1037C000894601456315D60023AE070405451C4311
:1037D00081CB97D70100938727D89843784315E387
:1037E000828097D60100938626D7904294427442F5
:1037F000850674C2E9B797D701009387E7D59C4344
:103800007DB7984394437C43FD177CC3FC42E9FB9E
:103810007360043082805D71A6C2CAC052DC56DA81
:103820005AD85ED686C6A2C44EDE62D466D26AD0AC
:1038300017D90100130949D317DB0100130B0BD271
:1038400097D401009384C4D197DA0100938A8AD176
:10385000054AA54B83270900984363010712DC47FB
:1038600083A90700EFE06FF6EFE02FF783270B0047
:103870002A8C6362F50A97D7010023A1A7CE0146DF
:103880006370351B8840B3858941EFD07FA2EFE09C
:10389000DF98630105128840814601462C00EFD075
:1038A000CFDB4DD9A247E3C807FEC24983A7490130
:1038B00089C713854900EFC0BFCBEFE00FF2832724
:1038C0000B002A8C636DF508A24717D70100232748
:1038D00087C9E3E2FBFCB317FA0013F70721631A69
:1038E000071613F7770C6318071E93F70702C5D75F
:1038F0004E85EF00F01145B7DC47C04783AC0700A9
:10390000930944004E85EFC0BFC65C502285829764
:103910005C4C6384470B83270900984371FF03A71E
:103920000A0097D6010023AB86C397D6010023ABCC
:10393000F6C297D7010023A9E7C2EFE01F8EA1BF0F
:10394000DC47C04703AD0700930C44006685EFC019
:103950003FC25C50228582975C4C6386470983276F
:103960000900984371FF03A70A0097D6010023AB13
:10397000F6BE97D7010023A9E7BEB9B7EFE0EFE4A1
:10398000EFE0AFE583270B002A8CE366F5F883A709
:103990000A00884081499043B385894117D70100C7
:1039A000232E87BB13361600EFD09F90EFE0FF86E3
:1039B000E31305EEEFC09FA5F9BD1C4CCE85E6973D
:1039C00063E9FC049C4089CF02CA66CC22CEEFF0AA
:1039D0000FE88840814601464C08EFD0EF8705FD8F
:1039E0007370043001A01C4CE685EA97636CFD04FB
:1039F0009C4089CF02CA6ACC22CEEFF04FE58840C6
:103A0000814601464C08EFD02F8531F973700430A0
:103A100001A0032509005CC000C8EFC07FB2E5BD6E
:103A2000EFE0AFFF83270900DC47C047930C440059
:103A30006685EFC0FFB35C4C638F47035C50228503
:103A4000829791BD032509005CC000C8EFC05FAF3D
:103A500039B7B24723ACF900A5CFE29723A2F9000A
:103A600023A8390193854900636FFC0403A50A006C
:103A7000EFC01FAD0DB51C4C00C83387F90058C00E
:103A8000636DEC02330C3C416363FC029C4089CFC4
:103A900002CA4ECC22CEEFF08FDB88408146014631
:103AA0004C08EFC07FFB59F97370043001A003A5E7
:103AB0000A00E685EFC0DFA851B703250900E685B7
:103AC000EFC01FA8A5BF03250900EFC07FA7E1B382
:103AD0007370043001A0B24783A6890123A839017D
:103AE0003387D70023A2E9006364EC04B307FC40EA
:103AF00063EBD70483A749024E85829783A7C90148
:103B0000E39B47D983A68901B2479840B69711CF66
:103B100002CA3ECC4ECEEFF08FD38840814601469C
:103B20004C08EFC07FF3E31805D67370043001A092
:103B30006374FC00E370F7FC0325090093854900DA
:103B4000EFC01FA089BB03A50A0093854900EFC001
:103B50003F9F91B3411122C406C626C24AC017D462
:103B600001001304E49FEFF04FE31C4095CBEFF00E
:103B70000FE51C409DC381480148814709478146A4
:103B80001306004097D50100938545831705000073
:103B90001305A5C8EFD05F9A39E97370043001A00E
:103BA00017D90100130989BC4A85EFC05F9697D4E5
:103BB00001009384E4BC2685EFC07F950146B145A2
:103BC000114597D7010023A1279B97D7010023AB6D
:103BD0009798EFC0FFC217D701002323A79811CDF4
:103BE00097C501009385057DEFD04FE149B7B240FD
:103BF000224492440249410182807370043001A042
:103C0000A5C9797156CAAA8A1305C00222D426D240
:103C10004AD04ECE52CC06D65AC85EC63A89B6892C
:103C2000328AAE84E9212A8405C9EFF00FD797D7ED
:103C300001009387E7929C439DCFEFF04FD8130587
:103C400044002320540104CC232E440123203403B8
:103C500023222403EFC0FF8C2285B25022549254B9
:103C60000259F249624AD24A424BB24B45618280C4
:103C70007370043001A097DB0100938B2BAF5E853E
:103C8000EFC0FF8817DB0100130B8BAF5A85EFC025
:103C90001F880146B145114597D7010023A6778DAE
:103CA00097D7010023A0678DEFC09FB517D70100FC
:103CB0002328A78A01C997C501009385A56FEFD076
:103CC000EFD3A5BF7370043001A039C5011122CC18
:103CD00006CE26CA17D40100130484888328040062
:103CE0002A88014563850802BA842EC2368732C409
:103CF00042C6954663C5B602EFF06FB58947630BC0
:103D0000F5020840814601464C00EFC0FFD4F24066
:103D10006244D244056182807370043001A04C007B
:103D200081463A864685EFC09FF5F2406244D24410
:103D3000056182800840814626864C00EFC0DFD1B5
:103D4000F9B719C1084182807370043001A001E500
:103D50007370043001A0411106C622C42A84EFF01A
:103D6000CFC348483334A000EFF06FC52285B2407E
:103D700022444101828001E57370043001A04111A9
:103D800022C42A8406C6EFF04FC10050EFF02FC3C3
:103D9000B240228522444101828001E573700430E3
:103DA00001A0411122C426C22E84AA8406C6EFF0C7
:103DB000CFBE80D02244B240924441016FF02FC068
:103DC0004111714522C406C61D262A8411C523202F
:103DD00005001105EFC0AFF32285B2402244410136
:103DE000828001CDB70700FFED8F81C7737004306B
:103DF00001A099E57370043001A07370043001A034
:103E0000011122CC4AC84EC652C456C206CE26CA9A
:103E1000BA893689B28A2E842A8AEFF04FA311E537
:103E2000638509007370043001A0EFE00F9A8324CA
:103E30000A00B37794006316090295C763870A00E6
:103E40009347F4FFE58F2320FA00EFE00FBDF24027
:103E5000624426854249D244B249224A924A0561C7
:103E60008280E30DF4FCE38209FEB3355001E205E4
:103E700063050900B7070004DD8D4E86C18D13056B
:103E80004A00EFE0FFE6EFE04FB919E1EFC00FD8CD
:103E9000EFF0CFB593176500AA8963D80700B70480
:103EA0000001FD14B3F499005DB7EFF00FAF832963
:103EB0000A00B3773401631E090089CB63880A00C6
:103EC0009347F4FFB3F737012320FA00EFF02FAF49
:103ED000F9B7E31DF4FEDDB701C9B70700FFED8FA9
:103EE00099C77370043001A07370043001A04111B0
:103EF00022C42A8406C626C24AC02E89EFF0EFA942
:103F000004409345F9FFB3F795001CC0EFF02FABC9
:103F1000B2402244268502499244410182804111E7
:103F200022C42A8406C6EFC04FDA0040EFC08FD902
:103F3000B240228522444101828009C9370700FF2F
:103F4000B3F7E50099C77370043001A073700430B3
:103F500001A06F20A05AB70700FFF18F81C77370CF
:103F6000043001A001E67370043001A0011122CCDD
:103F70004AC84EC652C406CE26CA3689AE892A8A97
:103F80003284EFF0CF8C21E16305090073700430B7
:103F900001A0EFE08F8383240A00CE855285B3E42D
:103FA0009900613FB37794006307F40683240A0005
:103FB000EFE0AFA6F240624426854249D244B249BE
:103FC000224A05618280EFE04F8083240A00CE857B
:103FD0005285B3E434019537B3F78400638D8702CB
:103FE000E30609FCB70500054A86C18D13054A00A2
:103FF000EFE01FD0EFE06FA219E1EFC02FC1EFF0AB
:10400000EF9E93176500AA8463DF0700B7070001DE
:10401000FD17FD8C45B783270A001344F4FFE18F99
:104020002320FA0071B7EFF04F9783240A00B3778B
:104030009400639787009347F4FFE58F2320FA00ED
:10404000EFF0EF97E1B7411122C406C62A8426C2D9
:10405000EFD0BFF75C4085C308489304C4006316E3
:10406000950015A0084863009502B7050002EFE02F
:104070003FE55C40E5FB2285612A2244B240924440
:1040800041016FE08F997370043001A009C93707AF
:1040900000FFB3F7E50099C77370043001A0737097
:1040A000043001A06F20804501C9B70700FFED8FE4
:1040B00099C77370043001A07370043001A04111DE
:1040C00022C426C206C62A84AE84EFF00F8D1840A3
:1040D00093C7F4FFF98F1CC02244B24092444101BF
:1040E0006FF0EF8D19C1084D82800145828041112A
:1040F00022C406C62A84EFD05FED97C701009387DC
:10410000E7469C43A1EBE56717C701001307C768A3
:10411000F11797C6010023A1E64617C70100232B1C
:10412000F74417C70100232BF76697C70100938751
:10413000274417C701002321F766854717C70100E9
:10414000232E074217C701002324074217C7010087
:10415000232EF74019E8EFE04F8CEF10C007014421
:104160002285B24022444101828013058400937766
:104170003500C1EFE5671307F5FFE917E3EDE7FC4D
:1041800097C601009386463F9C4229A0984311C7D9
:10419000BE86BA87D843E36BA7FE17C70100130793
:1041A000273DE38AE7FA984341461384870098C283
:1041B000D843B306A7406378D6023388A7002322EA
:1041C000D800C8C38325480097C601009386C63A25
:1041D00011A0BA8698425043E36DB6FE2320E80052
:1041E00023A00601D84397C701009387A73B9C43B0
:1041F000998F17C701002327F73AEFE00F8231DCD0
:104200002285B240224441018280719911059DB7F7
:1042100029C9411122C406C62A84EFD01FDB9305A9
:1042200084FF0326C4FF17C701001307E73411A05A
:104230003E871C43D443E3EDC6FE232CF4FE0CC39F
:1042400097C701009387073698438327C4FF22440A
:10425000B240BA9717C701002326F73441016FD047
:10426000DFFB828097C701009387C7338843828032
:1042700082803367B5000D8BAA871DE79308D6FFB0
:10428000AA982A87AE866371150303A80600110752
:104290009106232E07FFE36A17FF9347F5FFC697A2
:1042A000F19B9107BE95AA972A9663F3C70A938656
:1042B000450013884700B3B6D70033B8050133E78C
:1042C000F50093C61600134818000D8BB3E60601DF
:1042D00013371700758F330EF6409386170029CFDA
:1042E0001337AE0031EB13532E002E88BE860147E4
:1042F000832808000507110823A016019106E36929
:1043000067FE1377CEFFBA95BA976302EE0483C6B1
:104310000500138717002380D700637AC70283C67E
:10432000150013872700A380D7006372C70203C755
:1043300025002381E7008280B307F640AE9785050C
:1043400003C7F5FF8506238FE6FEE39AF5FE82801C
:104350008280B367C5008D8BB308C500E9C3637164
:10436000150FB307A0408D8B13873700954693F543
:10437000F50F130815003383A8407D166373D7002B
:1043800015476363E60CD5CF2300B5000547638D61
:10439000E700A300B5000D47130825006396E7006A
:1043A000130835002301B500139685004D8E139731
:1043B0000501518F3303F34093968501D98E13562F
:1043C0002300AA97014794C305079107E36DC7FE31
:1043D0001377C3FFB307E8006307E3062380B70042
:1043E00013871700637C1703A380B7001387270088
:1043F000637617032381B7001387370063701703B1
:10440000A381B70013874700637A17012382B7009F
:104410001387570063741701A382B700828093F556
:10442000F50F13978500D98D139705014D8FE3770D
:1044300015FFAA87910723AEE7FEE3ED17FF828001
:1044400082802A8895B78280AA8749BF8347050062
:104450002A8799C7050583470500EDFF198D8280DE
:104460000145828005058347F5FF850503C7F5FFF4
:1044700091C7E389E7FE3385E74082808147E5BF46
:10448000AA87850503C7F5FF8507A38FE7FE75FBA0
:10449000828083460500930700026397F6000505B6
:1044A00083460500E38DF6FE938756FD93F7D70FFD
:1044B00085C7AA87814585CE01458507138606FDF8
:1044C0001317250083C607003A9506053295F5F6C1
:1044D00099C13305A0408280938536FD834615003F
:1044E00093B5150093071500E1FA0145D5B70145CD
:1044F00082809C412380A7009C4185079CC18280CB
:1045000097C601009386C6079C42175703001307FE
:10451000672B13861700BA972380A70097C5010061
:1045200023A0C506A9476308F500930700046305A7
:10453000F6000145828075DE370610F005078347D7
:10454000F7FF2320F6F09C42FD1797C5010023A931
:10455000F502EDF7014582804D712322911423204D
:104560002115232A511323248113232611142324D4
:104570008114232E3113232C411323286113232666
:104580007113232291132320A113232EB111AA8486
:104590002E8932C6130C5002A54A83470900638056
:1045A0008703B9CB804011A0A1CB2300F400804049
:1045B0000509050480C083470900E39787FF034688
:1045C000190093081900C686130D0002FD597D5A83
:1045D0000148130550059307D6FD93F7F70F13898C
:1045E00016006363F52A17C701001307A7A18A07FE
:1045F000BA979C43BA9782878320C11403248114FD
:1046000083244114032901148329C113032A81132C
:10461000832A4113032B0113832BC112032C811214
:10462000832C4112032D0112832DC11171618280EF
:10463000A14C02C4854763D50715B2478040938BD0
:10464000770093F68BFF03AB060083A946009387A0
:1046500086003EC6668681465A85CE85EF10900458
:104660002AC8814763853723930D4101854B6686B0
:1046700081465A85CE85EF102025814666862A8B95
:10468000AE89EF103002A24723A0AD0093861B0035
:10469000910D63843701B68BD9BFE37E9BFF63DD49
:1046A0004601A2872380A70180407D1A930714004A
:1046B0009CC03E84E3C846FF93962B001C08BE9620
:1046C00031A8938777052300F4008040FD1B938772
:1046D0001B00050480C0F116E351F0EC9C42E3E2BC
:1046E000FAFE93870703C5B79C4093060003324741
:1046F0002380D7009C4093064700C14C13861700C7
:1047000090C013068007A380C700804002C4BA8708
:10471000050480C003AB0700814936C625BFB247F8
:1047200083AC0700938B470063840C1C635F4019C4
:104730009307D0026319FD1683C70C0085C363DCA1
:1047400009189440850C7D1A2380F60080400504EA
:1047500080C083C70C00E5F7635D4001804093078C
:1047600000022300F40080407D1A050480C0E31A93
:104770000AFE5EC61DB502C48547A94CE3CF07EB10
:10478000B24780409386470071B703C61600CA86B9
:1047900099B59C40930650022380D70080400504C1
:1047A00080C0E5BBC14C02C471B5B24703C6160058
:1047B000CA8683A9070091073EC6E35E0AE04E8AD7
:1047C000FD5911BD03C61600130DD002CA8621B5CE
:1047D0009347FAFFFD8703C61600337AFA00CA86AC
:1047E000DDBB03C61600130D0003CA86EDB383C5F7
:1047F0001600930906FDCA86938705FD2E86E3EE13
:10480000FAFA93972900BE9985068609AE9983C561
:104810000600938909FD938705FD2E86E3F3FAFED2
:1048200069BF32479C40144311073AC62380D70022
:104830008040050480C095B3854763D3070BB2471A
:1048400093867700E19A938786003EC683A9460047
:104850009C4263DC090A94401306D002B307F0407F
:104860002380C6008040B336F000B3093041050410
:1048700080C03E8BB389D940A94C02C4E1BB03C6BA
:1048800016000508CA8681BB9C40468921B7E37D96
:104890009BDD8547814B8546E3C547E131BD97CC1C
:1048A0000100938C2CB2CE856685EF00302A330A46
:1048B000AA40635C400180402300A40180407D1A2F
:1048C000050480C0E31A0AFE014A83C70C00E38294
:1048D00007EAE3C809E6FD197D57E394E9E6ADBDB3
:1048E000B247938647009C4336C693D9F74195B7A4
:1048F000635640019307D002E313FDFA97CC010001
:10490000938C4CAC930780021DBD3E8BA94C02C416
:10491000804089B34D71232E3113B709004093872E
:10492000F9FF2324811423229114232C4113232AD9
:104930005113232611142320211523286113232624
:10494000711323248113232291132320A113232ED7
:10495000B1112A8A2EC417C40100130464C2975AE5
:104960000300938A2AE697B401009384247F3EC60D
:1049700093055002294513080004B70610F0834739
:104980000A006386B704C1C71840050A130617005A
:10499000569797C8010023A5C8BE2300F70063827D
:1049A000A706E31E06FD175703001307A7E1050737
:1049B0008347F7FF23A0F6F01C40FD1717C6010040
:1049C0002320F6BCEDF783470A00E39EB7FA83463F
:1049D0001A0013051A002A87930B00027D5B7D5C89
:1049E000014893055005A5489387D6FD93F7F70F27
:1049F000130A170063E7F5348A07A6979C43A69726
:104A00008287175703001307E7DB55F28DBF83201A
:104A1000C11403248114832441140329011483291C
:104A2000C113032A8113832A4113032B0113832B00
:104A3000C112032C8112832C4112032D0112832DEC
:104A4000C11171618280A14C014D854763DB07195B
:104A5000A2479D07E19B83AD070003AB4700138787
:104A600087003AC4668681466E85DA85EF108043FA
:104A70002AC863066D35130941018549668681465A
:104A80006E85DA85EF00506466868146AA8D2E8B8E
:104A9000EF1040412320A90085091109E3106DFFA3
:104AA000E3FE9DFD13060004B70610F063D18903F1
:104AB0001C4013871700D69797C5010023A2E5ACC9
:104AC00023807701630CC7047D1CE3C389FFB247D1
:104AD0006800A548B386F9008A061C08BE962948D6
:104AE00013030004370610F0E384A6E89C42930504
:104AF000000363F4F800930570051840AE97930522
:104B00001700569717CE0100232CBEA62300F700EE
:104B10006380072B638C6526F116F9B717570300DE
:104B2000130747CA05078347F7FF23A0F6F01C4089
:104B3000FD1797C5010023A5F5A4EDF77D1C71B7FE
:104B40001C40130600041387170097C5010023A912
:104B5000E5A2B386FA00930500032380B600630F35
:104B6000C73C890797C6010023ACF6A05697930669
:104B700080072300D700175703001307A7C4B70601
:104B800010F0639EC70005078347F7FF23A0F6F0E8
:104B90001C40FD1717C601002324F69EEDF7A2471F
:104BA000C14C014D91072247014B832D07003EC4A4
:104BB00055BDA24783AC070013894700638E0C3AAA
:104BC000635480219307D002639EFB2E03C70C0021
:104BD000BA856310072025AC8547A94C014DE3C970
:104BE00007E7A2479107C1B7A2478346170052873C
:104BF00003AB070091073EC4E3580CDE5A8C7D5B83
:104C0000E5B383461700930BD0025287F1BB93475D
:104C1000FCFFFD8783461700337CFC005287E9B315
:104C200083461700930B000352877DBB0346170092
:104C3000138B06FD5287930706FDB286E3EEF8FA62
:104C400093172B00DA9705078607B29703460700EC
:104C5000138B07FD930706FDB286E3F3F8FE69BFE9
:104C6000A2451C402946984193861700D69717C540
:104C700001002327D5902380E700138945006300B6
:104C8000C72A930700046387F6204AC4D5B1854735
:104C900063DE0729A24713877700619B930787008C
:104CA0003EC4032B47001C43635A0B3018401306C5
:104CB00000049306170097C5010023A3D58C5697CF
:104CC0009305D0022300B7006387C62CB307F040DA
:104CD0003337F000330B6041BE8D330BEB40A94CF2
:104CE000014D49B38346170005085287F5B983463D
:104CF00017005287D5B91C4093060004138717008C
:104D000017C60100232EE686D6971306500223808D
:104D1000C700E31FD7C4175703001307A7AAB70696
:104D200010F005078347F7FF23A0F6F01C40FD179E
:104D300017C601002326F684EDF71DB9C14C014DBD
:104D400029B31C40930600042A8A1387170017C64C
:104D500001002327E682D697130650022380C7005E
:104D6000E318D7C0175703001307C7A5B70610F0FD
:104D700005078347F7FF23A0F6F01C40FD1717B681
:104D80000100232FF67EEDF72A8ADDB617570300C0
:104D9000130747A305078347F7FF2320F6F01C40BE
:104DA000FD1797B5010023ADF57CEDF7F1162DBB8E
:104DB00017570300130707A1F1FDF11635B3E3FC04
:104DC0009DCB8549C5B1014C03C70C00BA85E30EE4
:104DD00007EAFD58294513080004B70610F0635789
:104DE0000B0A1C4013861700D69717B3010023291E
:104DF000C3782380E7006384A50663040609850C55
:104E000003C70C007D1CBA8579FBE35080E91C4088
:104E10009305000213060004B70610F021A07D1CC4
:104E2000E3050CE613871700D6972380B70017B564
:104E300001002327E574BA87E313C7FE1757030061
:104E40001307479805078347F7FF23A0F6F01C4098
:104E5000FD1717B501002325F572EDF7C9B71757F0
:104E600003001307279641DE05078347F7FF23A0BA
:104E7000F6F01C40FD1717B601002323F670EDF77E
:104E8000BDBF175703001307E793F9BF7D1BE31A54
:104E90001BF5A5BF175703001307C792B70610F0FD
:104EA00005078347F7FF23A0F6F01C40FD1717B650
:104EB00001002327F66CEDF74AC45DBC97BC0100E6
:104EC000938C4C50DA8566855121330CAC40E35D00
:104ED00080EF1C4013060004B70610F021A07D1CD3
:104EE000E3030CEE13871700D6972380770197B55D
:104EF000010023A7E568BA87E313C7FE175703002D
:104F00001307478C05078347F7FF23A0F6F01C40E3
:104F1000FD1797B5010023A5F566EDF7C9B717573B
:104F200003001307278ABDFA4AC499B4A24713871E
:104F300047009C433AC413DBF741BDB31757030046
:104F400013074788B70610F005078347F7FF23A02C
:104F5000F6F01C40FD1717B601002323F662EDF7AB
:104F6000854717B70100232DF76093078007175770
:104F700003002309F78425B1635680019307D0020B
:104F8000E39EFBF297BC0100938CCC431307800295
:104F9000930580023DBD975603009386A68237068F
:104FA00010F0850603C7F6FF2320E6F018407D17B2
:104FB00097B5010023A6E55C6DF709BBBE8DA94C32
:104FC000014D4DB4B70710F023A0A7F201A039712D
:104FD000130341022ED29A8506CE32D436D63AD861
:104FE0003EDA42DC46DE1AC63532F2400145216126
:104FF00082805D711303810322D42AC632DC2A84A5
:105000001A86680006D6BEC236DEBAC0C2C4C6C69C
:105010001ACEEFF06FD4B247238007003245B2506A
:10502000018D225461618280B70710F083A647F496
:1050300003A607F403A747F4E31AD7FE8566938611
:1050400006FAB29633B6C600B305E60023A4D7F439
:1050500023A6B7F48280B70710F003A747F403A68E
:1050600007F483A647F4E31AD7FE8566938606FA0B
:10507000B29633B6C60023A4D7F4B305E60023A640
:10508000B7F49307000873A047308280411122C40F
:1050900006C629447D14312C75FCB24022444101DE
:1050A0008280411122C406C697B701009387C74D7D
:1050B00017B401001304044D98431C401306F07C00
:1050C000930647069387470697B5010023AED54A56
:1050D00097B5010023A8F54A6346D600B2402244A2
:1050E000410182801307478997B7010023AEE74843
:1050F0001D2485476310F502184085679387F7766E
:105100000145E3DDE7FCEFF0FFEB2244B240410153
:105110006FC0BFEA17B501001305452BEFF03FEB59
:105120000945EFF03FEA2244B24041016FC0FFE879
:1051300017B501001305052B6FF07FE917B50100C6
:105140001305C52A6FF0BFE8411122C426C206C666
:10515000856417B401001304E4299387843801009F
:10516000FD17F5FF2285EFF09FE6C5BF411106C68A
:1051700022C4DD2017070000130787F1814605468A
:105180009305200317B5010013054527EFE05FA73E
:105190002A84EFC09FE42A8622852244B240014738
:1051A0008146854541016FE05FB2411106C6A522E7
:1051B000054781476316E500B2403E854101828084
:1051C00017B5010013058520EFF07FE0B240894755
:1051D0003E85410182807370043001A0828073702B
:1051E000043001A0797122D426D24AD04ECE52CCBE
:1051F00006D6014917B401001304443A97B90100D7
:105200009389C93A17BA0100130A0A39854408403C
:105210008145EFC02FAA65DD814601466C00EFB0E5
:10522000DFC36306950097B7010023A10738B24793
:105230006382270397B7010023AA073683A70900D3
:10524000E39797FC83270A00850717B701002325FA
:10525000F73475BF0509DDB7411101469145294570
:1052600006C622C4EFB0CFD917B4010013044433EB
:1052700008C02945EFC0AF94AA870840BE8517B77C
:105280000100232DF730EFC04F9C2244B2408148EB
:1052900001488147014781461306004097B5010048
:1052A0009385051717050000130505F441016FC02C
:1052B000AFA897B701009387E72D9C4313072003FE
:1052C00085076367F70017B701002325F72C828055
:1052D000411197B701009387A72C06C688438146E2
:1052E000014697B501009385A52A97B7010023A32E
:1052F000072AEFB0DF988547631CF50097B70100D8
:10530000938707299C43850717B701002322F728B5
:10531000B2404101828097B701009387E72717B712
:1053200001001307A7269C4318436316F70017B71D
:105330000100232D072617B701001307272708436D
:1053400017B701002324F72482800000B305B500BD
:10535000930705006386B70003C7070063160700BD
:105360003385A74067800000938717006FF09FFE8A
:10537000130101FB23229104232C410323229103D7
:10538000232611042324810423202105232E310305
:10539000232A510323286103232671032324810335
:1053A0002320A103232EB101930C0500138A0500CD
:1053B0009304000063DE05003305A0403337A000EE
:1053C000B305B040930C0500338AE5409304F0FF29
:1053D00063DA06003306C040B337C000B306D040DE
:1053E000B386F640930A06009389060013840C00E6
:1053F00013090A006396062817BB0100130B8BEBF9
:105400006370CA16B70701006372F6149307F00FB2
:1054100063F4C70093098000B3573601330BFB00D8
:1054200083470B0013050002B3873701B309F5402A
:10543000638C0900B3153A01B3D7FC00B31A3601E7
:1054400033E9B70033943C0113DB0A0193050B00E9
:1054500013050900EF00507C130A050093050B00AB
:10546000939B0A0113050900EF00907693DB0B0173
:105470009305050013850B00EF00D072131A0A0183
:1054800093570401B367FA0063FAA700B387570183
:1054900063E6570163F4A700B38757013389A74038
:1054A00093050B0013050900EF001077130A0500A0
:1054B00093050B0013050900EF009071131404010C
:1054C00093050500131A0A0113850B0013540401F8
:1054D000EF00506D33648A00637AA40033045401F2
:1054E000636654016374A400330454013304A4407C
:1054F0003354340193050000638A04003304804070
:10550000B3378000B305B040B385F5401305040000
:105510008320C1040324810483244104032901045A
:105520008329C103032A8103832A4103032B010337
:10553000832BC102032C8102832C4102032D010223
:10554000832DC1011301010567800000B707000129
:1055500093090001E362F6EC930980016FF0DFEB41
:10556000631A06009305000013051000EF00506653
:10557000930A0500B707010063FAFA0E9307F00FCC
:1055800063F4570193098000B3D73A01330BFB0052
:1055900083470B001305000233095A41B3873701D3
:1055A000B309F540E38209EAB39A3A01335BFA00A2
:1055B000B3153A01B3D7FC0093DB0A0133E9B70016
:1055C00013050B0093850B00EF001065130A05000F
:1055D00093850B00139C0A0113050B00EF00505F2D
:1055E000135C0C019305050013050C00EF00905BA4
:1055F000131A0A0193570901B367FA0033943C0167
:1056000063FAA700B387570163E6570163F4A70065
:10561000B3875701338BA74093850B0013050B000D
:10562000EF00905F130A050093850B0013050B0034
:10563000EF00105A9305050013050C00EF0090567B
:1056400093160901131A0A0193D60601B366DA000C
:1056500063FAA600B386560163E6560163F4A6001A
:10566000B38656013389A6406FF01FDEB7070001ED
:1056700093090001E3EAFAF0930980016FF0DFF08B
:105680006376DA0093050A006FF01FE7B7070100A1
:1056900063FAF604930BF00F33B5DB0013153500F6
:1056A00033D7A60097B701009387C7C0B387E70039
:1056B00083CB070093050002B38BAB00338B75419E
:1056C000631C0B0263E4460163EACC003384CC40E4
:1056D000B306DA4033B98C003389264193050900BB
:1056E0006FF09FE1B707000113050001E3EAF6FA46
:1056F000130580016FF0DFFAB3966601335D760122
:10570000336DDD00B35D7A01B3156A0133DC7C01D2
:1057100013540D01336CBC0013850D009305040078
:10572000B3196601EF00504F930A0500930504007A
:1057300013850D0033996C01931C0D01EF00504946
:1057400093DC0C01130A05009305050013850C007A
:10575000EF005045939A0A0113570C0133E7EA0012
:10576000930D0A00637EA7003307A701930DFAFF8C
:105770006368A7016376A700930DEAFF3307A701CB
:10578000330AA7409305040013050A00EF00D04830
:1057900093050400930A050013050A00EF00504327
:1057A000930505001304050013850C00EF00903FDE
:1057B00093150C01939A0A0193D50501B3E5BA003C
:1057C0001307040063FEA500B385A5011307F4FFCA
:1057D00063E8A50163F6A5001307E4FFB385A501FF
:1057E000939D0D01B70C0100B3EDED001384FCFF98
:1057F000B3F78D0033F48900338AA5401385070081
:10580000930504002326F10093DD0D01EF0090398C
:1058100093050400930A050013850D00EF009038EE
:1058200013DC090193050C002324A10013850D004E
:10583000EF0050378327C10013040C0093050400C8
:10584000130C050013850700EF00D0358326810077
:1058500013D70A013305D5003307A7006374D700B7
:10586000330C9C01B70701009387F7FF935507019D
:105870003377F70013170701B3F7FA00B3858501F3
:10588000B307F7006366BA00631EBA00637CF900D1
:1058900033863741B3B7C700B385A541B385F5401B
:1058A00093070600B307F9403339F900B305BA404E
:1058B000B385254133947501B3D767013364F40090
:1058C000B3D565016FF05FC3130101FD232291027F
:1058D000232A51012326110223248102232021039C
:1058E000232E3101232C410123286101232671013C
:1058F00023248101232291012320A101930A050081
:1059000093840500639E063813040600930905007E
:1059100017B901001309099A63F8C512B707010006
:10592000138B05006378F6101307F00F3337C700A9
:1059300013173700B357E6003309F900834609000F
:105940003387E60093060002B386E640638C0600C8
:10595000B394D40033D7EA003314D600336B9700E6
:10596000B399DA00935A040193850A0013050B00DA
:10597000EF00902A1309050093850A00931B040188
:1059800013050B00EF00D02493DB0B0193040500FB
:105990009305050013850B00EF00D02013190901B2
:1059A00093D70901B367F900138A040063FEA700C7
:1059B000B3878700138AF4FF63E8870063F6A700C4
:1059C000138AE4FFB3878700B384A74093850A0056
:1059D00013850400EF0050241309050093850A0085
:1059E00013850400EF00D01E93990901930405006C
:1059F000930505001319090113850B0093D90901BB
:105A0000EF00501AB36939011386040063FCA90042
:105A1000B30934011386F4FF63E6890063F4A90037
:105A20001386E4FF13140A013364C400130A000050
:105A30006F000013B707000113070001E36CF6EED7
:105A4000130780016FF01FEF138A0600631A060028
:105A50009305000013051000EF00901713040500D4
:105A6000B7070100637EF4129307F00F63F4870019
:105A7000130A8000B35744013309F90003470900B2
:105A80009306000233074701B386E640639406128B
:105A9000B3848440130A1000135B040193050B00C8
:105AA00013850400EF0050171309050093050B0040
:105AB00013850400931B0401EF00901193DB0B018D
:105AC000930405009305050013850B00EF00900D6E
:105AD0001319090193D70901B367F900938A0400E8
:105AE00063FEA700B3878700938AF4FF63E887000B
:105AF00063F6A700938AE4FFB3878700B384A740C7
:105B000093050B0013850400EF0010111309050025
:105B100093050B0013850400EF00900B9399090186
:105B200093040500930505001319090113850B0063
:105B300093D90901EF001007B369390113860400F6
:105B400063FCA900B30934011386F4FF63E68900FE
:105B500063F4A9001386E4FF13940A013364C400BC
:105B60001305040093050A008320C1020324810267
:105B700083244102032901028329C101032A8101EF
:105B8000832A4101032B0101832BC100032C8100D7
:105B9000832C4100032D01001301010367800000E5
:105BA000B7070001130A0001E366F4EC130A800151
:105BB0006FF05FEC3314D40033DAE400B399DA0009
:105BC00033D7EA00935A0401B394D40093850A00B2
:105BD00013050A00336B9700EF001004130905004A
:105BE00093850A0013050A00931B0401EF00407E11
:105BF00093DB0B01930405009305050013850B004F
:105C0000EF00407A1319090113570B013367E900BC
:105C1000138A0400637EA70033078700138AF4FF0A
:105C2000636887006376A700138AE4FF3307870061
:105C3000B304A74093850A0013850400EF00C07DDC
:105C40001309050093850A0013850400EF004078CE
:105C5000930405009305050013850B00EF00807485
:105C600013170B011357070113190901B367E90053
:105C70001387040063FEA700B38787001387F4FF30
:105C800063E8870063F6A7001387E4FFB387870004
:105C9000131A0A01B384A740336AEA006FF0DFDF0A
:105CA00063ECD51EB707010063F4F6041307F00F89
:105CB000B335D7009395350033D7B60097A70100C9
:105CC0009387475FB387E70003C70700130A000203
:105CD0003307B700330AEA4063160A0213041000C0
:105CE000E3E096E833B6CA00134416006FF05FE7AE
:105CF000B707000193050001E3E0F6FC930580017E
:105D00006FF09FFBB35CE600B3964601B3ECDC009A
:105D100033D4E40093DB0C01B397440133D7EA009A
:105D200093850B0013050400336BF700B31946018C
:105D3000EF00806E1309050093850B001305040026
:105D4000139C0C01EF00C068135C0C019304050068
:105D50009305050013050C00EF00C0641319090139
:105D600013570B013367E90013840400637EA70017
:105D7000330797011384F4FF636897016376A700E4
:105D80001384E4FF33079701B304A74093850B0006
:105D900013850400EF0040681309050093850B008C
:105DA00013850400EF00C06293040500930505000D
:105DB00013050C00EF00005F93170B011319090185
:105DC00093D70701B367F9001386040063FEA700A9
:105DD000B38797011386F4FF63E8970163F6A70082
:105DE0001386E4FFB387970113140401B70B010076
:105DF0003364C4001389FBFF337D240133F9290187
:105E0000B384A7409305090013050D00EF008059E6
:105E1000935C040193050900130B050013850C0026
:105E2000EF00405893D90901130C05009385090030
:105E300013850C00EF000057130905009385090036
:105E400013050D00EF0000563305850193570B0134
:105E50003385A700637485013309790193570501E0
:105E6000B387270163E6F402E392F4BCB7070100AD
:105E70009387F7FF3375F50013150501337BFB009E
:105E800033964A0133056501130A0000E37AA6CC74
:105E90001304F4FF6FF09FB9130A0000130400000D
:105EA0006FF01FCC130101FB2324810423229104F2
:105EB000232E3103232291032326110423202105BD
:105EC000232C4103232A5103232861032326710332
:105ED000232481032320A103232EB101930C050069
:105EE000938905001304050093840500639E06262C
:105EF00013090600138A060097AA0100938A8A3BB9
:105F000063F4C514B70701006376F6129307F00F28
:105F100063F4C700130A8000B3574601B38AFA003E
:105F200003C70A001305000233074701330AE5409F
:105F3000630C0A00B395490133D7EC0033194601CD
:105F4000B364B70033944C01935A090193850A0056
:105F500013850400EF00404C9309050093850A0067
:105F6000131B090113850400EF008046135B0B012E
:105F70009305050013050B00EF00C042939909013A
:105F800093570401B3E7F90063FAA700B387270129
:105F900063E6270163F4A700B3872701B384A74012
:105FA00093850A0013850400EF000047930905005C
:105FB00093850A0013850400EF0080411314040147
:105FC000930505009399090113050B00135404016F
:105FD000EF00403D33E48900637AA40033042401D8
:105FE000636624016374A400330424013304A440D1
:105FF00033554401930500008320C1040324810428
:1060000083244104032901048329C103032A810352
:10601000832A4103032B0103832BC102032C81023A
:10602000832C4102032D0102832DC10113010105BF
:1060300067800000B7070001130A0001E36EF6EC69
:10604000130A80016FF05FED631A060093050000EC
:1060500013051000EF00C03713090500B707010052
:10606000637AF90E9307F00F63F42701130A800097
:10607000B3574901B38AFA0003C70A0013050002A7
:10608000B384294133074701330AE540E30E0AEAA6
:1060900033194901B3DAE900B395490133D7EC006C
:1060A00093540901336BB70013850A0093850400EC
:1060B000EF0080369309050093850400931B0901C6
:1060C00013850A00EF00C03093DB0B019305050038
:1060D00013850B00EF00002D9399090193570B01D5
:1060E000B3E7F90033944C0163FAA700B3872701A3
:1060F00063E6270163F4A700B3872701B38AA740AB
:106100009385040013850A00EF0000319309050010
:106110009385040013850A00EF00802B930505008A
:1061200013850B00EF00002893150B0193990901CB
:1061300093D50501B3E5B90063FAA500B385250140
:1061400063E6250163F4A500B3852501B384A5406A
:106150006FF09FDFB7070001130A0001E36AF9F04F
:10616000130A80016FF0DFF0E3E8D5E8B70701001C
:1061700063FCF604930BF00F33B5DB001315350009
:1061800033D7A60097A701009387C712B387E7000C
:1061900083CB070093050002B38BAB00338B7541B3
:1061A000631E0B0263E4360163EACC003384CC4007
:1061B000B386D94033B58C00B384A64013050400E0
:1061C000938504006FF05FE3B7070001130500013A
:1061D000E3E8F6FA130580016FF09FFAB3966601C3
:1061E000335D7601336DDD0033D47901B3956901F8
:1061F00033DC7C0193540D01336CBC0013050400A7
:1062000093850400B31A6601EF000021130A05000C
:10621000938504001305040033996C01931C0D0150
:10622000EF00001B93DC0C0113040500930505002F
:1062300013850C00EF000017131A0A0113570C0105
:106240003367EA00130A0400637EA7003307A7013F
:10625000130AF4FF6368A7016376A700130AE4FF3B
:106260003307A701B309A7409385040013850900EC
:10627000EF00801A938504001304050013850900BC
:10628000EF000015930505009304050013850C002D
:10629000EF00401193150C011314040193D505016F
:1062A000B365B4001387040063FEA500B385A501A0
:1062B0001387F4FF63E8A50163F6A5001387E4FFE5
:1062C000B385A501131A0A01B70C0100336AEA006D
:1062D0001384FCFFB3778A0033F48A00B384A540AB
:1062E00013850700930504002326F100135A0A01C1
:1062F000EF00400B930905009305040013050A0005
:10630000EF00400A13DC0A01930D050093050C0011
:1063100013050A00EF0000098327C100130A0500D6
:1063200093050C0013850700EF00C0073305B50186
:1063300013D709013307A7006374B701330A9A0121
:10634000B70701009387F7FF935507013377F700ED
:1063500013170701B3F7F900B3854501B307F70039
:1063600063E6B400639EB400637CF9003386574152
:10637000B3B7C700B385A541B385F54093070600C1
:10638000B307F9403339F900B385B440B3852541EB
:1063900033947501B3D767013365F400B3D5650154
:1063A0006FF09FC5130605001305000093F6150056
:1063B000638406003305C50093D515001316160037
:1063C000E39605FE678000006340050663C6050688
:1063D00013860500930505001305F0FF630C060204
:1063E00093061000637AB6006358C00013161600B7
:1063F00093961600E36AB6FE1305000063E6C50037
:10640000B385C5403365D50093D6160013561600E4
:10641000E39606FE6780000093820000EFF05FFBCA
:1064200013850500678002003305A04063D805008E
:10643000B305B0406FF0DFF9B305B04093820000C0
:10644000EFF01FF93305A04067800200938200003F
:1064500063CA0500634C0500EFF09FF71385050044
:1064600067800200B305B040E35805FE3305A04045
:10647000EFF01FF63305B0406780020097A70100D8
:106480009387870D944317A701001307A70B1843A1
:10649000C8C2637BE50017A701001307670B084319
:1064A0008C4391056FA0CF89411122C406C617A75E
:1064B00001001307270A2A8408438C439105EFA0A3
:1064C0002F8897A70100938727069C436376F400E3
:1064D00097A7010023AA8704B24022444101828089
:1064E00097A7010093874707984394437C43FD1780
:1064F0007CC3FC4299E3736004308280011122CC9A
:1065000026CA2A84AE844AC84EC652C456C206CE93
:10651000EFB0BFAB1C4003290401B7090001B3E58C
:106520009700930AC4000CC08144FD19370A000289
:106530001840638C2A03032609004A85B365470186
:10654000B376360193175600758F0329490063C44B
:10655000070001E7F1BFE39DE6FC9317760063D3E4
:106560000700D58CEFC0DF95E1B793C4F4FFF98C39
:1065700004C0EFB09FCA0840F2406244D24442498E
:10658000B249224A924A05618280411106C622C45C
:10659000EFE0DFBD17F7FFFF1307E7B081460546C1
:1065A0009305400617A501001305C5E5EFD04FE59B
:1065B00019C92A84EFB07FA22A8601478146854502
:1065C0002285EFD08FF0EFB0CFFAB24022440145E0
:0465D0004101828083
:02000004800278
:100000008A47FEFF8848FEFF9247FEFF8848FEFFB2
:100010008848FEFF8848FEFF8848FEFFAA47FEFF8B
:100020008848FEFF8848FEFFC447FEFFD047FEFF1A
:100030008848FEFFE247FEFFEE47FEFFEE47FEFF69
:10004000EE47FEFFEE47FEFFEE47FEFFEE47FEFFE8
:10005000EE47FEFFEE47FEFFEE47FEFF8848FEFF3D
:100060008848FEFF8848FEFF8848FEFF8848FEFF5C
:100070008848FEFF8848FEFF8848FEFF8848FEFF4C
:100080008848FEFF8848FEFF8848FEFF8848FEFF3C
:100090008848FEFF8848FEFF8848FEFF8848FEFF2C
:1000A0008848FEFF8848FEFF8848FEFF8848FEFF1C
:1000B0008848FEFF8848FEFF8848FEFF8848FEFF0C
:1000C0008848FEFF8848FEFF8848FEFF8848FEFFFC
:1000D0008848FEFF8848FEFF8848FEFF8848FEFFEC
:1000E0008848FEFF8848FEFF8848FEFF8848FEFFDC
:1000F0008848FEFF8848FEFF8848FEFF8848FEFFCC
:100100002248FEFF3848FEFF8848FEFF8848FEFF71
:100110008848FEFF8848FEFF8848FEFF8848FEFFAB
:100120008848FEFF7E48FEFF8848FEFF8848FEFFA5
:100130003046FEFFE846FEFF8848FEFF8848FEFF87
:100140001E47FEFF8848FEFF7647FEFF8848FEFFF9
:100150008848FEFFA447FEFF964BFEFFEA4BFEFFDA
:100160009E4BFEFFEA4BFEFFEA4BFEFFEA4BFEFF13
:10017000EA4BFEFF904AFEFFEA4BFEFFEA4BFEFF12
:10018000AA4AFEFFB64AFEFFEA4BFEFFC84AFEFF40
:10019000D44AFEFFD44AFEFFD44AFEFFD44AFEFFF3
:1001A000D44AFEFFD44AFEFFD44AFEFFD44AFEFFE3
:1001B000D44AFEFFEA4BFEFFEA4BFEFFEA4BFEFF8E
:1001C000EA4BFEFFEA4BFEFFEA4BFEFFEA4BFEFF67
:1001D000EA4BFEFFEA4BFEFFEA4BFEFFEA4BFEFF57
:1001E000EA4BFEFFEA4BFEFFEA4BFEFFEA4BFEFF47
:1001F000EA4BFEFFEA4BFEFFEA4BFEFFEA4BFEFF37
:10020000EA4BFEFFEA4BFEFFEA4BFEFFEA4BFEFF26
:10021000EA4BFEFFEA4BFEFFEA4BFEFFEA4BFEFF16
:10022000EA4BFEFFEA4BFEFFEA4BFEFFEA4BFEFF06
:10023000EA4BFEFFEA4BFEFFEA4BFEFFEA4BFEFFF6
:10024000EA4BFEFFEA4BFEFFEA4BFEFFEA4BFEFFE6
:10025000EA4BFEFFEA4BFEFF084BFEFF364BFEFF6C
:10026000EA4BFEFFEA4BFEFFEA4BFEFFEA4BFEFFC6
:10027000EA4BFEFFEA4BFEFFEA4BFEFF8C4BFEFF14
:10028000EA4BFEFFEA4BFEFFEE48FEFFE849FEFFA9
:10029000EA4BFEFFEA4BFEFF5A4AFEFFEA4BFEFF27
:1002A000804AFEFFEA4BFEFFEA4BFEFFE44BFEFFF7
:1002B000000102020303030304040404040404040D
:1002C00005050505050505050505050505050505DE
:1002D00006060606060606060606060606060606BE
:1002E00006060606060606060606060606060606AE
:1002F000070707070707070707070707070707078E
:10030000070707070707070707070707070707077D
:10031000070707070707070707070707070707076D
:10032000070707070707070707070707070707075D
:10033000080808080808080808080808080808083D
:10034000080808080808080808080808080808082D
:10035000080808080808080808080808080808081D
:10036000080808080808080808080808080808080D
:1003700008080808080808080808080808080808FD
:1003800008080808080808080808080808080808ED
:1003900008080808080808080808080808080808DD
:1003A00008080808080808080808080808080808CD
:1003B000546D725100000000546D7220537663003A
:1003C000286E756C6C2900004572726F7220696E20
:1003D00020787878207461736B73200D0A00000018
:1003E0006D69616F750A00006D69616F75320A0091
:1003F00068756E6772790A0054696D657232000023
:10040000436865636B54696D657200005365745091
:040410006F6C6C00A1
:100414001000000000000000017A5200017C01017C
:100424001B0D02005000000018000000404FFEFFAA
:100434005805000000440E507489039406990B81FA
:1004440001880292049305950796089709980A9AD9
:100454000C9B0D036C010AC144C844C944D244D363
:1004640044D444D544D644D744D844D944DA44DBAC
:10047400440E00440B0000004C0000006C0000001F
:100484004454FEFFDC05000000440E3070890395DF
:1004940007810188029204930594069608970998A7
:1004A4000A990B9A0C0370020AC144C844C944D285
:1004B40044D344D444D544D644D744D844D944DA64
:1004C400440E00440B00000050000000BC0000007B
:1004D400D059FEFF0005000000440E5074880289C4
:1004E400039305990B810192049406950796089746
:1004F40009980A9A0C9B0D0320010AC144C844C9F7
:1005040044D244D344D444D544D644D744D844D91B
:0C05140044DA44DB440E00440B000000FD
:0C05A000FC8F01000900000001000000B9
:040000058000004037
:00000001FF
